:100026000A0A54657374696E6720314220506F72F4
:100036007420285033342C50313729202E2E2E0090
:100046000A5479706520616E79206B657973207426
:100056006F2065786974000A0A54657374696E675F
:1000660020334220506F727420285033322C503384
:10007600332C5033352C5031302C5031312C5031FB
:100086003429202E2E2E000A0A54657374696E6771
:1000960020492F4F20506F727420285031322C5037
:1000A60031332C50313729202E2E2E000A0A546562
:1000B6007374696E672031324220506F7274202843
:1000C60050312C5033322C5033332C5033342C5087
:1000D600333529202E2E2E000A0A54657374696E54
:1000E600672032344220506F7274205B38323535C7
:1000F6002F453030302D45303033485D202E2E2EA2
:10010600000A0A54657374696E67204C4344205094
:100116006F72742077697468204C434432307832A9
:1001260020284261636B6C696768742D50433429DB
:10013600202E2E2E000A0A54657374696E672034C9
:1001460078384B2C3878384420506F72742026202B
:10015600537065616B657220283832353529202E3B
:100166002E2E000A0A54657374696E6720494E5430
:10017600302C494E5431204B657920262044697035
:100186002D537769746368202E2E2E000A494E542B
:10019600302C494E542C446970312D34203D2000BA
:1001A600300031000A0A54657374696E6720525430
:1001B6004320445331333037202E2E2E000A5479F3
:1001C60070652028532920746F2073657420746924
:1001D6006D652061742032333A35393A353520322F
:1001E600382F30322F3034000A6F7220616E79203A
:1001F6006B65797320746F20436F6E74696E7565D5
:1002060020446973706C6179203A000A74696D65DF
:100216002025303262783A25303262783A253032FB
:1002260062782020646174652025303262782F253B
:10023600303262782F2530326278000A0A546573AC
:1002460074696E6720454570726F6D2032344C4379
:100256003034202E2E2E20004572726F722021001F
:100266004F4B000A5479706520616E79206B657971
:1002760073200054657374696E672052414D2025C2
:100286003034582D2530345848202E2E2E0A00257D
:100296003034582020202000253034583D4F4B2044
:1002A600000A0A000A0A426C616E6B2D300A000AC7
:1002B6000A426C616E6B2D310A000A0A426C616E4D
:1002C6006B2D320A000A0A426C616E6B2D330A00EE
:1002D6000A0A54657374696E672032344220506F7F
:1002E6007274205B492F4F2D383235352D435331EB
:1002F6005D202E2E2E000A0A54657374696E6720DF
:1003060032344220506F7274205B492F4F2D3832A1
:1003160035352D4353325D202E2E2E000A0A5465A4
:100326007374696E67204C434420506F7274207753
:10033600697468204C434432307832202842616325
:100346006B6C696768742D50323729202E2E2E006B
:100356000A0A54657374696E6720494E54302C49F5
:100366004E5431204B6579202620537065616B65AC
:1003760072202850333529202E2E2E000A494E543D
:10038600302C494E54203D20000A0A576F726B6983
:100396006E67202E2E2E000A0A4261636B6C696717
:1003A6006874203D204F4E000A0A4261636B6C69F7
:1003B600676874203D204F4646000A0A54657374E8
:1003C6002045582D536572696573202832344220C2
:1003D600506F72742C5041302D504133206F722073
:1003E6005041342D50413729202E2E2E000A5479A3
:1003F600706520302D3720746F20776F726B200068
:100406000A0A546573742045582D536572696573DD
:10041600202831324220506F72742C5031302D50CA
:100426003133206F72205031342D50313729202E30
:100436002E2E000A0A546573742045582D53657292
:100446006965732028334220506F72745B503130D7
:100456002C5031312C5031335D20262053657420C9
:10046600416464726573732041302D41323D3029F9
:10047600202E2E2E000A0A546573742044502D53E4
:1004860065726965732028334220506F72745B5021
:1004960031302C5031312C5031335D2C36423539C8
:1004A600352C382044696769747329202E2E2E0056
:1004B6000A576F726B696E6720000A0A5465737477
:1004C6002044502D536572696573202833422050AD
:1004D6006F72745B5031302C5031312C5031335D9A
:1004E6002C6D6178373231392C382044696769744C
:1004F6007329202E2E2E000A0A54657374696E67BE
:100506002044502C444B2D53657269657320285343
:1005160063616E20387838442C3478384B20506F1D
:10052600727429202E2E2E000A0A54657374696E81
:100536006720525332333220746F20334220506F7B
:1005460072742053657269616C2028544C434429A7
:10055600202E2E2E000A54797065204374726C2D5D
:100566004320746F206578697420000A0A54657305
:1005760074204D61676E657469632C50726F78697B
:100586006D6974792028334220506F72745B503144
:10059600302C5031312C5031335D29202E2E2E0A2D
:1005A600002563000A0A5465737420534854313594
:1005B6002054656D7020262048756D6964697479CC
:1005C6002028334220506F72745B5031302C5031EA
:1005D600312C5031335D29202E2E2E000A54253021
:1005E600352E316620482530342E3166000A0A53EE
:1005F600656C65637420313D4D3438543038203293
:100606003D4D3438543335203E000A5465737469C1
:100616006E6720525443204D343854787820284F42
:100626006E20444D454D20303030304820536F63A6
:100636006B6574292E2E2E004F4B0D0045520D0072
:100646004552002530326258000D00253032626472
:100656000D002530326278253032627825303262DC
:10066600780D0025303262580D00534C41422D352D
:10067600312076342E330D00542530352E31662048
:10068600482530342E31660D000A00534C41422D68
:1006960035312051432050726F6772616D20763478
:1006A6002E3320283839563531524432424E290AE3
:1006B60000436865636B73756D3D25303458205370
:1006C600706565643D25750A003230303620536901
:1006D6006C6120526573656172636820436F2E2CCE
:1006E6004C74642E000A5479706520616E79206B13
:1006F600657973202E2E2E002020202323232320ED
:100706005465737420457870616E73696F6E20420C
:100716006F6172642023232323200A00312E204593
:10072600582D536572696573202832344220506F04
:1007360072742C416374697665204869676829205C
:100746000A00322E2045582D53657269657320289C
:1007560031324220506F72742C4163746976652081
:100766004C6F7729200A00332E2045582D53657289
:100776006965732028334220506F72742C4163746C
:10078600697665204C6F772C49324329200A00345C
:100796002E2044502D5365726965732028334220FC
:1007A600506F72742C364235393529200A00352EA1
:1007B6002044502D536572696573202833422050BA
:1007C6006F72742C4D61783732313929200A003620
:1007D6002E2044502C444B2D536572696573202896
:1007E6005363616E20387838442C3478384B205067
:1007F6006F727429200A00372E205253323332206A
:10080600746F20334220506F727420536572696191
:100816006C2028544C434429200A00512E2051753F
:100826006974200A0020202053656C656374203AA1
:1008360000070020202023232323205465737420DF
:100846004C4344204D6F64756C652023232323207D
:100856000A00312E20444D43303832200A00322E11
:1008660020444D43313631200A00332E20444D4377
:10087600313632200A00342E20444D43313634209E
:100886000A00352E20444D43323032200A00362EDF
:1008960020444D43323034200A00372E2042616313
:1008A6006B6C69676874204F6E2F4F6666200A006E
:1008B600202020232323232054657374204163635F
:1008C6006573736F7279202620436F6D706F6E6546
:1008D6006E742023232323200A00312E204D6167C6
:1008E6006E657469632C50726F78696D69747920CE
:1008F6000A00322E2053485431352054656D70203D
:10090600262048756D6964697479200A00332E20A3
:10091600525443204D34385430382C4D34385433E7
:1009260035200A002020202323232320534C414234
:100936002D35312076342E33204D656E75202323D8
:10094600232320202020202020534C41422D3531C6
:1009560020562D433531353520562D433532200A64
:1009660000202020202020202020202020202020A1
:100976002020202020202020202020202020202071
:10098600202020202020202076342E3020202020D9
:1009960076352E3020202076332E30200A00312E58
:1009A60020314220506F727420285033342C50313D
:1009B6003729202E2E2E2E2E2E2E2E2E2E2E2E2E5B
:1009C6002E2E2E2E2E2058200A00322E2033422084
:1009D600506F727420285033322C5033332C5033DE
:1009E600352C5031302C5031312C50313429202EB9
:1009F6002E2058202E2E2E2E2E2058202E2E2E2EF5
:100A06002058200A00332E20492F4F20506F727431
:100A160020285031322C5031332C50313729202E9A
:100A26002E2E2E2E2E2E2E2E2E2E2E2E2E2E2E2EE0
:100A36002E2E2E2E2058202E2E2E2E2058200A0006
:100A4600342E2031324220506F7274202850312CBF
:100A56005033322C5033332C5033342C5033352909
:100A6600202E2E2E2E2E2E2058202E2E2E2E2E20AE
:100A760058202E2E2E2E2058200A00352E203234B5
:100A86004220506F72742028453030302D38323570
:100A96003529202E2E2E2E2E2E2E2E2E2E2E2E2E7C
:100AA6002E2E2058202E2E2E2E2E2058200A00368E
:100AB6002E204C434420506F72742028433030302F
:100AC6002D4261636B6C696768742D50433429202D
:100AD6002E2E2E2E2E2E2058200A00372E20347829
:100AE600384B2C3878384420506F727420262053A7
:100AF6007065616B657220283832353529202E2EB7
:100B06002E2E2058200A00382E20494E54302C49CB
:100B16004E5431204B65792026204469702D537739
:100B260069746368202E2E2E2E2E2E2E2E2E2058E1
:100B3600200A00392E205254432044533133303793
:100B4600202E2E2E2E2E2E2E2E2E2E2E2E2E2E2ECD
:100B56002E2E2E2E2E2E2E2E2E2E2058202E2E2EA1
:100B66002E2E2E2E2E2E2E2E2E2058200A00412ED0
:100B760020454570726F6D2032344C433034202E40
:100B86002E2E2E2E2E2E2E2E2E2E2E2E2E2E2E2E7F
:100B96002E2E2E2E2E2058202E2E2E2E2E2E2E2E61
:100BA6002E2E2E2E2058200A00422E2052616D2015
:100BB600303030302D31464646482028384B2920E3
:100BC6002E2E2E2E2E2E2E2E2E2E2E2E2E2E2E2E3F
:100BD6002058202E2E2E2E2E2058200A00432E205E
:100BE60052616D20303030302D3746464648202839
:100BF60033324B29202E2E2E2E2E2E2E2E2E2E2EFC
:100C06002E2E2E2E2058202E2E2E2E2E2058200A06
:100C160000442E2052616D20303030302D3746464C
:100C2600464820283132384B292033327834204246
:100C36006C616E6B202E2E2E2E2E2E2E2E2E2E2EEE
:100C46002058200A00452E2052616D203830303061
:100C56002D39464646482028384B29202E2E2E2E42
:100C66002E2E2E2E2E2E2E2E2E2E2E2E2058202E90
:100C76002E2E2E2E2058200A00462E2032344220B8
:100C8600506F72742028492F4F2D383235352D4339
:100C9600533129202E2E2E2E2E2E2E2E2E2E2E2E59
:100CA6002E2E2E2E2E2E2E2E2E2E2E2E2E2E2E206C
:100CB60058200A00472E2032344220506F7274208A
:100CC60028492F4F2D383235352D43533229202EC2
:100CD6002E2E2E2E2E2E2E2E2E2E2E2E2E2E2E2E2E
:100CE6002E2E2E2E2E2E2E2E2E2E2058200A004848
:100CF6002E204C434420506F72742028492F4F2DCC
:100D06004261636B6C696768742D50323729202EF7
:100D16002E2E2E2E2E2E2E2E2E2E2E2E2E2E2E2EED
:100D26002E2E2E2E2E2058200A00492E20494E54B3
:100D3600302C494E5431204B65792026205370655E
:100D4600616B6572202850333529202E2E2E2E2ECB
:100D56002E2E2E2E2E2E2E2E2E2E2E2E2E2E2E2EAD
:100D66002058200A00582E20546573742045787048
:100D7600616E73696F6E20426F617264200A00595A
:100D86002E2054657374204C4344204D6F64756C5B
:100D960065200A005A2E20546573742041636365EA
:100DA60073736F7279202620436F6D706F6E656E58
:100DB60074200A00E0E1E2E3E4E5E6E7D0D1D2D32D
:100DC600D4D5D6D7B0B1B2B3B4B5B6B77071727365
:100DD600747576773F065B4F666D7D077F6F777C10
:100DE600395E79717E306D79335B5F707F7B771FFB
:040DF6004E3D4F47D8
:074B7900AF8E4307028F8E8F
:014B80002212
:074B8100AF8E5307FD8F8E7C
:014B8800220A
:10434300852782852683EAF0A3F085278285268345
:07435300A3A3F07F587E02D6
:10435A00EF4E60147D737C00ED1D70011CED4C70F6
:08436A00F7EF1F70EB1E80E865
:014372002228
:10475E00EFC394614006EFD39466400CEFC39441CF
:10476E00400BEFD394465005EF24098001EF540F10
:02477E00FF2218
:0C494600786CE6FF12475EAE0718E6FF33
:0949520012475EEFC454F0FF228D
:1020CF00758910E4F58DF58BC28E20B0FDD28EA2EE
:1020DF00B0B340FBC28EAF8DAB07EBFAAF8BEFFB0C
:1020EF00E47F64FE12435A7F20D3EB94E4EA941109
:1020FF00400AEB940CEA941250028060D3EB94E800
:10210F00EA9408400AEB9410EA940950028065D3D0
:10211F00EB946AEA9404400AEB9492EA9404500216
:10212F00806AD3EB942CEA9402400AEB9454EA941D
:10213F00025002806FD3EB940CEA9401400BEB94A6
:10214F0034EA940150030221DC7F3AD3EB94EAEA9C
:10215F009405400FEB9412EA9406500775570475D7
:10216F0058B022D3EB94ECEA9402400FEB9414EAAC
:10217F009403500775570975586022D3EB946CEA96
:10218F009401400FEB9494EA940150077557127520
:10219F0058C022D3EB94ACEA9400400FEB94D4EAEE
:1021AF009400500775572575588022D3EB944CEA4D
:1021BF00940040047E0180027E00C3EB9474EA9485
:1021CF000050047D0180027D00ED5E600775574B66
:0E21DF00755800227F647E0012435A0220CF02
:103F1100759852758920E5588557F01213F33F378C
:103F210004B03F3C09603F4112C03F4625803F4BF2
:103F31004B0000003F51758DE88015758DF48010A0
:103F4100758DFA800B758DFD8006758DFD4387801B
:033F5100D28E22EB
:0A4AFD007F057E0012435AD2B42256
:084B89003018FD0000C2B42247
:1040C600C209E4FFFE7DFF7C4F20090B8D828C83A5
:1040D600E493F46002D20930090B8D828C83E49359
:1040E6002FFFE43EFEED1D70011CED4C70DB9000D1
:0840F60000E4932FFFE43EFEFD
:0140FE00229F
:0D4ABF0090C000EFF090C001E020E7F92268
:0C48D10074FF2EF582E434FFF583E0FF55
:0D48DD0090C002EFF090C001E020E7F9224A
:104A4800E4FE7F38124ABF0EBE04F77F0C024ABF4D
:03495B00124A48B5
:10495E007F01124ABF7F509000007420F0A3DFFC4D
:01496E002226
:1022EE00E559640170257F80124ABF7E011248D1E4
:1022FE000EBE09F97FC0124ABF7E0174072EF58209
:10230E00E434001248D90EBE09F122E55964057075
:10231E00517F80124ABF7E011248D10EBE15F97F41
:10232E00C0124ABF7E0174132EF582E434001248A7
:10233E00D90EBE15F17F94124ABF7E0174272EF579
:10234E0082E434001248D90EBE15F17FD4124ABF72
:10235E007E01743B2EF582E434001248D90EBE1570
:10236E00F1227F80124ABF7E01EED3955A5006129B
:10237E0048D10E80F4E5646401605D7FC0124ABFEF
:10238E007E01EED3955A500E74132EF582E434006E
:10239E001248D90E80ECE5646402603C7F90124ACC
:1023AE00BF7E01EED3955A500E74272EF582E4347B
:1023BE00001248D90E80ECE5646403601B7FD012D6
:1023CE004ABF7E01EED3955A500E743B2EF582E431
:0823DE0034001248D90E80EC16
:0123E60022D4
:102EAF00E5596401701EAE63EEC3940850074306E4
:102EBF0080AF06806FEEC394105071EE24F844C0BB
:102ECF00FEFF8060E5596405702EE56770047E8013
:102EDF008019E567B401047EC08010E567B4020471
:102EEF007E948007E567B403027ED4E563C3955AE9
:102EFF00503AE5632EFF802CE56770047E808019C1
:102F0F00E567B401047EC08010E567B402047E90CB
:102F1F008007E567B403027ED0E563C3955A500C72
:0C2F2F00E5632EFF124ABF7F0E124ABF5E
:012F3B002273
:10498300C2A4C2A5D2A68F80C2A6D2A67F017E00F2
:0349930002435A82
:0F478000AF030B74002FF582E43400F583E0FFE4
:10478F00D2A4C2A5D2A68F80C2A6D2A67F017E00D8
:03479F0002435A78
:104A5800E4FB7F381249830BBB04F77F0C024983C0
:1049E2007F011249837F289000007420F0A3DFFC2E
:0149F20022A2
:10480500E4FB7F801249837A011247800ABA15F9C1
:0E4815007FC01249837A011247800ABA15F952
:014823002272
:10417100D3ED9400EC64809480402C90D002E05404
:10418100BFF07E01EED39F5008ED1D70011C0E8023
:10419100F390D002E04440F07E01EED39F50D1ED88
:0741A1001D70011C0E80F3EC
:0141A80022F4
:10458300D3ED9400EC648094804022C2B57E01EEAA
:10459300D39F5008ED1D70011C0E80F3D2B57E0130
:0D45A300EED39F50DBED1D70011C0E80F368
:0145B00022E8
:10392700C20AE4FB90D002E054F04BF9F074082B84
:10393700F8E690D000F07F017E0012435AE4F0A32E
:10394700E0540FF9640F6027D20A201622E9C45405
:10395700F04BF9E4FAEA900DBA93B5010E7DD07CED
:10396700077F14124171D216AF02220ABA20E60B62
:0A397700BB08B1200A02C2167FFF50
:013981002223
:0749F3007FDC7E0512435A30
:0949FA007F107808E4F608DFFCE8
:014A03002290
:0C4ACC00E4FE74082EF8A6070EBE08F6E3
:014AD80022BB
:064AD90054F0C4540FFF6D
:074ADF00EF900DDA93FF22B6
:074B9100EF900DEA93FF22F3
:094B430000000000000000002247
:054B9800D295024B4321
:054B9D00C295024B432C
:0E4A8700D296D295C296124B43C295D2962279
:0A4B0700C296D295124B43D29622BB
:07431200124A877FD07E00F4
:104319007D01EF339209A2099296EF25E0FFEE3372
:10432900FE124B98124B9D0DBD09E7D296124B9880
:09433900A2969209124B9DA20903
:014342002258
:10437300E4FF7E01124B98A2969209EF25E0FFA27B
:1043830009E4334207124B9D0EBE09E8D296124B45
:0F43930098A2969209124B9DA209B350027FFF88
:0143A20022F8
:10468100E4FF7E01124B98A2969209EF25E0FFA26A
:1046910009E4334207124B9D0EBE09E8C296124B44
:0646A10098124B9DD29619
:0146A70022F0
:0A4B110053187F531ABF531FEC2204
:03000300124B118C
:10000600124312E4FFFE124319E4FC74182CF8E6BE
:0D001600FF7E001243190CBC08F1024B07DD
:1042AE00124312E4FFFE124319124B07124B431234
:1042BE004A877FD17E00124319E4FD124681AC0776
:1042CE0074182DF8A6040DBD07F11243738F1F024B
:0242DE004B078C
:054BA200D295024B4317
:054BA700C295024B4322
:0E4A9500D296D295C296124B43C295D296226B
:0A4B1B00C296D295124B43D29622A7
:09424800AC07124A957FA07E002C
:104251007D01EF33920AA20A9296EF25E0FFEE3339
:10426100FE124BA2124BA70DBD09E7D296124BA22B
:09427100A296920A124BA7A20AC0
:01427A002221
:1043A300E4FF7E01124BA2A296920AEF25E0FFA240
:1043B3000AE4334207124BA70EBE09E8D296124B0A
:0F43C300A2A296920A124BA7A20AB350027FFF42
:0143D20022C8
:10482400AB05AA04124248AF047E00124251AF0302
:0F483400AE02124251124B1B7F057E0002435A07
:1043D300124248AF047E00124251124B1B7F017EF2
:1043E3000012435A124A957FA17E00124251124392
:0F43F300A3AB07124B1B7F017E0012435AAF038F
:014402002297
:1034F1008F828E83E04480F0E518547FA3F0E519B4
:10350100547F8F828E83A3A3F0E51A543F8F828E5E
:1035110083A3A3A3F0E51B5407FD74042FF582E4F4
:103521003EF583EDF0E51C543FFD74052FF582E473
:103531003EF583EDF0E51D541FFD74062FF582E481
:103541003EF583EDF074072FF582E43EF583E51E29
:09355100F08F828E83E0547FF0BC
:01355A00224E
:103982008F828E83E04440F0A3E0F5188F828E830D
:10399200A3A3E0F5198F828E83A3A3A3E0F51A7483
:1039A200042FF582E43EF583E0F51B74052FF582C2
:1039B200E43EF583E0F51C74062FF582E43EF583C0
:1039C200E0F51D74072FF582E43EF583E0F51E8FC6
:0739D200828E83E054BFF078
:0139D90022CB
:0E40FF00EAFD7C00E4FF12410D0F12410D0F8F
:10410D00EF14601014601314601624037016C2A10E
:10411D00C2A08010C2A1D2A0800AD2A1C2A08004E8
:0B412D00D2A1D2A08D80C2B6D2B62273
:054BAC00D2B3024B43EF
:054BB100C2B3024B43FA
:0E4AA300D2B5D2B3C2B5124B43C2B3D2B522C4
:0A4B2500C2B5D2B3124B43D2B52241
:1045B1007D01EF33920AA20A92B5EF25E0FFEE33B7
:1045C100FE124BAC124BB10DBD09E7D2B5124BAC8B
:0945D100A2B5920A124BB1A20A34
:0145DA0022BE
:10440300E4FF7E01124BACA2B5920AEF25E0FFA2B6
:104413000AE4334207124BB10EBE09E8D2B5124B80
:0F442300ACA2B5920A124BB1A20AB350027FFFAE
:014432002267
:1047A200AB078D828C83124AA3EB25E0540E447032
:1047B200FBFF7E001245B1AF82AE831245B1024BC0
:0147C20025D1
:1048EA00124AA3EF25E0540E4471FF7E001245B12F
:0648FA00124403124B25DD
:014900002294
:054BB600D291024B4307
:054BBB00C291024B4312
:0E4AB100D294D291C294124B43C291D294225D
:0A4B2F00C294D291124B43D294229B
:1045DB007D01EF33920AA20A9294EF25E0FFEE33AE
:1045EB00FE124BB6124BBB0DBD09E7D294124BB664
:0945FB00A294920A124BBBA20A21
:014604002293
:10443300E4FF7E01124BB6A294920AEF25E0FFA29D
:104443000AE4334207124BBB0EBE09E8D294124B67
:0F445300B6A294920A124BBBA20AB350027FFF8B
:014462002237
:1047C300AB078D828C83124AB1EB25E0540E447003
:1047D300FBFF7E001245DBAF82AE831245DB024B4B
:0147E3002FA6
:10490100124AB1EF25E0540E4471FF7E001245DBDF
:06491100124433124B2F8B
:01491700227D
:04446300AB05AA04F7
:104467007D01EF3392B5EF25E0FFD2B2C2B20DBDA9
:1044770009F07D01EB3392B5EB25E0FBEA33FAD285
:0B448700B2C2B20DBD09EDD2B3C2B34A
:014492002207
:10460500C2B2C2B3E4FDFC7F0F1244637D017F0C8F
:10461500124463E4FD7F09124463E556FD7F0A12E7
:0A4625004463E568FD7F0B02446367
:103E8700124605E508FD7C007F01124463E509FD44
:103E97007F02124463E50AFD7F03124463E50BFDCD
:103EA7007F04124463E50CFD7F05124463E50DFDB5
:103EB7007F06124463E50EFD7F07124463E50FFD9D
:053EC7007F08024463C6
:04449300AB05AA04C7
:104497007D01EF339294EF25E0FFD290C2900DBDDE
:1044A70009F07D01EB339294EB25E0FBEA33FAD276
:0B44B70090C2900DBD09EDD291C291A2
:0144C20022D7
:10462F00C290C291E4FDFC7F0F1244937D017F0C79
:10463F00124493E4FD7F09124493E556FD7F0A125D
:0A464F004493E568FD7F0B024493DD
:103ECC0012462FE508FD7C007F01124493E509FDA5
:103EDC007F02124493E50AFD7F03124493E50BFD28
:103EEC007F04124493E50CFD7F05124493E50DFD10
:103EFC007F06124493E50EFD7F07124493E50FFDF8
:053F0C007F0802449350
:10484300E4FF74502FF582E43400F583E4F07478C8
:0E4853002FF582E43400F583E4F00FBF28E473
:014861002234
:103ADB0020B5FDE4FFFEFDD20B20B54630B304301C
:103AEB00B5FA220000A2B2920A300B05200A02C2DC
:103AFB000BA20BB35027EFC313FF300A034307800E
:103B0B000EBE0519EF131313541FF4541FFF7450FB
:103B1B002DF582E43400F583EFF00DE4FE20B3B90C
:023B2B0080FB1D
:013B2D002275
:103B2E002094FDE4FFFEFDD20C209446309104302B
:103B3E0094FA220000A290920B300C05200B02C2C8
:103B4E000CA20CB35027EFC313FF300B03430780B7
:103B5E000EBE0519EF131313541FF4541FFF7450A8
:103B6E002DF582E43400F583EFF00DE4FE2091B9DB
:023B7E0080FBCA
:013B80002222
:10362800E4FE74502EF582E43400F583E0FF604731
:10363800E4FDFBEF13920BEFC313FF300B010D0BEF
:10364800BB05F0ED20E002D32274502EF582E4345D
:1036580000F583E0540FFFC3940A4008EF24F744B1
:1036680040FF800343073074782EF582E43400F578
:1036780083EFF00EBE28AB900078E064426002D37E
:0236880022C35B
:01368A00221D
:102831007D28900078E4F0A3DDFC7D28E4FCF9FB21
:10284100D20CEDD39400406A1D74502DF582E4340E
:1028510000F583E0FE300C0260E8EE33333354F8C8
:10286100FE7F01EFD3940550D9EE5480FAEE25E0B6
:10287100FEBA8004D20B8002C20B300C05300B0271
:10288100C20C200C2A300B05430480800353047FC3
:10289100ECC313FC0BBB05171313543FFCAB01092D
:1028A10074782BF582E43400F583ECF0E4FCFB0F43
:1028B10080B1EBD39400401EEB64056007ECC313B9
:1028C100FC0B80F4EC1313543FFC747829F582E47B
:1028D1003400F583ECF0E4FD74782DF582E43400E6
:1028E100F583E0FC74502DF582E43400F583ECF0BF
:0428F1000DBD28E40D
:0128F50022C0
:1041E000C2B2C2B3E4FFEFD3955C501F74082FF83E
:1041F000E6FEE4FDEE3392B5EE25E0FED2B200001D
:10420000C2B200000DBD08EC0F80DBD2B30000C2CB
:03421000B30000F8
:014213002288
:10421400C290C291E4FFEFD39555501F74082FF854
:10422400E6FEE4FDEE339294EE25E0FED29000002B
:10423400C29000000DBD08EC0F80DBD2910000C2DB
:03424400910000E6
:014247002254
:07488100C2B3124888D2B354
:104888000000000000000000000000000000000020
:054898000000000022F9
:1044C300E4FE7D80EDD394004017ED5F6004D2B22B
:1044D3008002C2B2D2B3124888C2B3EDC313FD80C7
:0F44E300E3D2B2D2B3124888A2B2E433C2B3FF1D
:0144F20022A7
:1044F300E4FED2B27D80EDD394004013D2B31248D0
:104503008830B203ED4206C2B3EDC313FD80E7EF7B
:0F45130024FF92B2D2B3124888C2B3D2B2AF061D
:014522002276
:10491800D2B2124881C2B2124888124881D2B21269
:074928004888C2B302488871
:10489D00D2B2C2B3124888E4FFD2B3124888C2B371
:0A48AD001248880FBF0AF2024918F2
:102D9300E4F5321249187F031244C3EF2532F532AA
:102DA300D2B2900000AF82AE83E4FCFD7B407A9CFC
:102DB300F9F8D31213A7400630B203A380E730B269
:102DC300020532E532D39400400BE4F536F535F5D0
:102DD30034F53380407F011244F3AB07EB7B00FAF9
:102DE3007F011244F3EFFBE4FF1244F3AE02AF039F
:102DF300AD07AC06E412106A7B0A7AD77923783CD4
:102E0300120EF2E4FBFA792078C2120E018F368E8D
:0D2E1300358D348C33AF36AE35AD34AC3375
:012E2000228F
:081D6F008F358E348D338C3268
:101D7700E4F536F544F5437542807541C07548541E
:101D87007547E375462575453D754CA2754BE77557
:101D97004A3B7549B675500A754FD7754E23754D31
:101DA7003C7554AC7553C57552A77551381249180F
:101DB7007F051244C3EF2536F536D2B2900000AF47
:101DC70082AE83E4FCFD7B407A9CF9F8D31213A71B
:101DD700400630B203A380E730B2020536E536D3BA
:101DE7009400400CE4F540F53FF53EF53D021F1623
:101DF7007F011244F37537008F38E538753800F5E1
:101E0700377F011244F3EF4238E4FF1244F3AC3753
:101E1700AD38E412106AAB4CAA4BA94AA849120E76
:101E2700F2C004C005C006C007AC37AD38E41210D5
:101E37006AD003D002D001D000120EF2C004C00550
:101E4700C006C007AC37AD38E412106AAB48AA47E2
:101E5700A946A845120EF2D003D002D001D0001235
:101E67000E01AB44AA43A942A841120E018F3C8E32
:101E77003B8D3A8C39AC37AD38E412106AAB54AAB3
:101E870053A952A851120EF2AB50AA4FA94EA84D12
:101E9700120E01C004C005C006C007E4FFFE7DC8DE
:101EA7007CC1AB35AA34A933A832120E01D003D0B6
:101EB70002D001D000120EF2AB3CAA3BA93AA839D6
:101EC700120E018F408E3F8D3E8C3DE4FFFE7DC894
:101ED7007C42AB40AA3FA93EA83D120FF8600F40D5
:101EE7000DE4F540F53F753EC8753D4280217FCD35
:101EF7007ECC7DCC7C3DAB40AA3FA93EA83D120FCE
:101F0700F8500C7540CD753FCC753ECC753D3DAF57
:071F170040AE3FAD3EAC3DC2
:011F1E0022A0
:10452300E4FE7D80EDD394004017ED5F6004D290EC
:104533008002C290D291124888C291EDC313FD80CC
:0F454300E3D290D291124888A290E433C291FF44
:014552002246
:10455300E4FED2907D80EDD394004013D2911248B3
:1045630088309003ED4206C291EDC313FD80E7EF5F
:0F45730024FF9290D291124888C291D290AF0645
:014582002216
:1046A800D290C291124888D291124888C29012487A
:1046B80088C291124888D291124888D290124888AC
:0546C800C291024888C8
:1048B700D290C291124888E4FFD291124888C291DF
:0A48C7001248880FBF0AF20246A84B
:102E2100E4F5321246A87F03124523EF2532F5322D
:102E3100D290900000AF82AE83E4FCFD7B407A9C8F
:102E4100F9F8D31213A74006309003A380E730901E
:102E5100020532E532D39400400BE4F536F535F541
:102E610034F53380407F01124553AB07EB7B00FA09
:102E71007F01124553EFFBE4FF124553AE02AF034E
:102E8100AD07AC06E412106A7B0A7AD77923783C45
:102E9100120EF2E4FBFA792078C2120E018F368EFF
:0D2EA100358D348C33AF36AE35AD34AC33E7
:012EAE002201
:081F1F008F358E348D338C32B6
:101F2700E4F536F544F5437542807541C07548546C
:101F37007547E375462575453D754CA2754BE775A5
:101F47004A3B7549B675500A754FD7754E23754D7F
:101F57003C7554AC7553C57552A77551381246A8D0
:101F67007F05124523EF2536F536D290900000AF56
:101F770082AE83E4FCFD7B407A9CF9F8D31213A769
:101F87004006309003A380E73090020536E536D34C
:101F97009400400CE4F540F53FF53EF53D0220C6C0
:101FA7007F011245537537008F38E538753800F5CE
:101FB700377F01124553EF4238E4FF124553AC37E0
:101FC700AD38E412106AAB4CAA4BA94AA849120EC5
:101FD700F2C004C005C006C007AC37AD38E4121024
:101FE7006AD003D002D001D000120EF2C004C0059F
:101FF700C006C007AC37AD38E412106AAB48AA4731
:10200700A946A845120EF2D003D002D001D0001283
:102017000E01AB44AA43A942A841120E018F3C8E80
:102027003B8D3A8C39AC37AD38E412106AAB54AA01
:1020370053A952A851120EF2AB50AA4FA94EA84D60
:10204700120E01C004C005C006C007E4FFFE7DC82C
:102057007CC1AB35AA34A933A832120E01D003D004
:1020670002D001D000120EF2AB3CAA3BA93AA83924
:10207700120E018F408E3F8D3E8C3DE4FFFE7DC8E2
:102087007C42AB40AA3FA93EA83D120FF8600F4023
:102097000DE4F540F53F753EC8753D4280217FCD83
:1020A7007ECC7DCC7C3DAB40AA3FA93EA83D120F1C
:1020B700F8500C7540CD753FCC753ECC753D3DAFA6
:0720C70040AE3FAD3EAC3D11
:0120CE0022EF
:103A3100D2B2D2B3E4FEEF30E704D2B58002C2B510
:103A41007C007D02ED1D70011CED4C70F7C2B27C53
:103A5100007D02ED1D70011CED4C70F7D2B2EF2517
:103A6100E0FF0EBE08D0C2B37C007D02ED1D7001E7
:103A71001CED4C70F7D2B37C007D14ED1D70011C60
:043A8100ED4C70F7A1
:013A8500221E
:103A8600D290D291E4FEEF30E704D2948002C29441
:103A96007C007D02ED1D70011CED4C70F7C2907C20
:103AA600007D02ED1D70011CED4C70F7D290EF25E4
:103AB600E0FF0EBE08D0C2917C007D02ED1D7001B4
:103AC6001CED4C70F7D2917C007D14ED1D70011C2D
:043AD600ED4C70F74C
:013ADA0022C9
:10427B007BFF7A0079261214827BFF7A0079461233
:10428B001482E4FB2098148B20A20092B4A201921A
:10429B00977FC87E0012435A0B80E9124B39D2B478
:0242AB00D297A8
:0142AD0022EE
:103DAE007BFF7A00795D1214827BFF7A00794612CE
:103DBE001482E4FB2098248B20A20092B2A20192DE
:103DCE00B3A20292B5A2039290A2049291A205927E
:103DDE00947F327E0012435A0B80D9124B39D2B2E5
:0A3DEE00D2B3D2B5D290D291D29494
:013DF80022A8
:104138007BFF7A00798D1214827BFF7A0079461210
:104148001482E4FB2098188B20A2039292A2049276
:1041580093A20592977F327E0012435A0B80E51294
:084168004B39D292D293D29799
:01417000222C
:103157007BFF7A0079B21214827B017528FE7527EE
:1031670001E5281313543F44C3F526852890852687
:10317700B07F907E0112435AE52825E04401F528E7
:103187000527E527D3940840D80BBB04CE75270144
:10319700752855E5281313543F44C3F52685289011
:1031A7008526B01243567528AAE5281313543F44C1
:1031B700C3F5268528908526B01243560527E527AF
:0B31C700D3940340CB7590FF75B0FF60
:0131D20022DA
:04380F008E268F274B
:103813008F828E83A3A3A37480F079017A017B0145
:10382300852782852683EAF0A3F085278285268370
:10383300A3A3F07F907E0112435AEA25E0FA0BBB63
:1038430009DE09B904D67B017A551243437AAA12D9
:1038530043430BBB04F2E4852782852683F0A3F060
:09386300852782852683A3A3F0CA
:01386C002239
:104A68007BFF7A0079DE1214827F007EE002380F25
:102FC8007BFF7A01790712148275590475640275BA
:102FD8005A1412495B7FE87E0312435A90D002E0EC
:102FE80054EFF07B30E4F52674002526F582E434AE
:102FF80000F583EBF00526E526B450EC1222EE7FAF
:10300800907E0112435A0BBB3ADBE4F52674002587
:1030180026F582E43400F58374FFF00526E526B42E
:1030280050EB1222EEE4F52690D002E054EFF07F48
:10303800C87E0012435AE04410F07FC87E00124355
:0A3048005A0526E526D3940340DE66
:01305200225B
:103C76007BFF7A01793B1214827BFF7A0079461228
:103C860014821249FA7F40124ACC20982F12392703
:103C96008F26E526F460F3E526124AD98F08E52635
:103CA600540FFF124ADF8F0985080A85080C85081C
:0F3CB6000E85090B85090D85090F80CE024B394C
:103332007BFF7A0179691214827BFF7A0079461247
:1033420014827527FF20985690D001E054F0FF13A5
:1033520013543FF52630B20343260130B30343260C
:1033620002E526652760DE7BFF7A017992121482DC
:10337200852628E4F529E5287BFF20E0067A0179F5
:10338200A680047A0179A8121482E528C313F528CD
:103392000529E529D3940540DD85262780A7024B20
:0133A20039F1
:103053007BFF7A0179AA1214827BFF7A0179C3126A
:1030630014827BFF7A0179EE121482124B39AB077B
:10307300EB64536003BB731F751C28751D02751E1B
:1030830004751B01751A2375195975185512000318
:103093007FC87E0012435A7BFF7A0079461214825E
:1030A3007BFF20982E7F647E0012435A1242AEE5C6
:1030B300186B60EE7BFF7A027911851A3585193614
:1030C300851837851C38851D39851E3A121482AB45
:0630D3001880CF024B390A
:103B81007BFF7A0279411214827DAA7C00E4FF1244
:103B910048247D557C007F01124824C209E4FF12AC
:103BA10043D3EF64AA6002D2097F011243D3EF64C9
:103BB100556002D2097BFF3009067A02795E8004E2
:103BC1007A0279661214827BFF7A02796912148271
:033BD100024B396B
:07269E007DFF7C7FE4FFFEDD
:0826A5008E268F278C288D2959
:1026AD007BFF7A027979852635852736852837850A
:1026BD002938121482124B7985262A85272B752EDF
:1026CD0011D3E52B9529E52A9528501D852B82855B
:1026DD002A83E52EF0052EE52EB49A03752E1105ED
:1026ED002BE52B70DC052A80D885262A85272B859E
:1026FD002A2C852B2D752E11C209D3E52B9529E595
:10270D002A9528504A852B82852A83E0652E600202
:10271D00D209852B82852A83E4F0052EE52E649A55
:10272D007023752E117BFF3009067A02799580048E
:10273D007A02799E852C35852D36121482C2098533
:10274D002A2C852B2D052BE52B70AF052A80AB127E
:0E275D004B817BFF7A027969121482024B399C
:104996007BFF7A0279A71214827DFF7C1FE4FFFE5B
:0349A6000226A541
:1049A9007BFF7A0279A71214827DFF7C7FE4FFFEE8
:0349B9000226A52E
:103DF900C296C2957BFF7A0279AA12148212269E74
:103E0900C296D2957BFF7A0279B512148212269E48
:103E1900D296C2957BFF7A0279C012148212269E2D
:103E2900D296D2957BFF7A0279CB1214827DFF7CE0
:073E39007FE4FFFE0226A555
:10496F007BFF7A0279A71214827DFF7C9F7F007EE6
:04497F00800226A5E7
:103E40007D807C007F0312410D79017A017B011294
:103E500040FF7F907E0112435AEA25E0FA0BBB092E
:103E6000EE09B904E67B017A551240FF1243567AF7
:103E7000AA1240FF1243560BBB04ECE4FAFDFCFF10
:073E80001241090F02410D80
:104A04007BFF7A0279D6121482C2A2123E40D2A24D
:014A1400227F
:104A15007BFF7A0279FC121482C2A3123E40D2A314
:014A2500226E
:1031D3007BFF7A037922121482124A581249E27F42
:1031E300E87E0312435AC2A77930E4F5267400251A
:1031F30026F582E43400F583E9F00526E526B4508C
:10320300EC1248057F907E0112435A09B93ADBE478
:10321300F52674002526F582E43400F58374FFF067
:103223000526E526B450EB124805E4F526C2A77F30
:10323300C87E0012435AD2A77FC87E0012435A05A4
:0832430026E526D3940340E5C3
:01324B002260
:103414007BFF7A0379561214827BFF7A0079461275
:1034240014827527FF209855E4F52630B20343260D
:103434000130B303432602E526652760E87BFF7A63
:10344400037982121482852628E4F529E5287BFF76
:1034540020E0067A0179A680047A0179A812148200
:10346400E528C313F5280529E529D3940140DD8512
:1034740026277D107C277F1412458380A8024B39B0
:1021ED007BFF7A03798F121482E5591460181460FD
:1021FD001A14601C14602114602324057025756465
:10220D0002755A08801D756401800875640280038B
:10221D00756404755A10800B75640280037564042F
:10222D00755A1412495B7FE87E0312435A7B30E4E2
:10223D00F52874002528F582E43400F583EBF005CC
:10224D0028E528B450EC1222EE7F907E0112435AFD
:10225D000BBB3ADBE4F52874002528F582E4340045
:10226D00F58374FFF00528E528B450EB1222EE7FBC
:10227D00E87E0312435A7B41E4F52874002528F5C6
:10228D0082E43400F583EBF00B0528E528B414EB5C
:10229D007B6175281474002528F582E43400F583DC
:1022AD00EBF00B0528E528B428EB7B417528287445
:1022BD00002528F582E43400F583EBF00B0528E5C5
:1022CD0028B43CEB7B6175283C74002528F582E42D
:1022DD003400F583EBF00B0528E528B450EB022212
:0122ED00EE02
:1046CD00B2147BFF30140F7A03799D12148290D0AF
:1046DD0002E054EFF0227A0379AE12148290D002E8
:0546ED00E04410F02282
:1025CF0090E0037480F0E4F5287BFF7A0379C01262
:1025DF0014827BFF7A0379F3121482124B39EF24A2
:1025EF00D0B40800400302269D90260675F003A480
:1025FF00C58325F0C5837302261E02262D02263CB5
:10260F0002264B02265A022669022678022687E501
:10261F002830E0055328FE806C4328018067E528A9
:10262F0030E1055328FD80034328028058E5283008
:10263F00E2055328FB80034328048049E52830E353
:10264F00055328F78003432808803AE52830E4052E
:10265F005328EF8003432810802BE52830E50553DE
:10266F0028DF8003432820801CE52830E605532807
:10267F00BF8003432840800DE52830E70553287FAE
:0E268F00800343288090E000E528F00225EA51
:01269D00221A
:10355B007590FF7BFF7A0479061214827BFF7A0346
:10356B0079F3121482124B39EF24D0B40800504671
:10357B0090358975F003A4C58325F0C58373023597
:10358B00A10235A50235A90235AD0235B10235B51B
:10359B000235B90235BDB29080CBB29180C7B292E1
:1035AB0080C3B29380BFB29480BBB29580B7B29602
:0635BB0080B3B29780AF5F
:0135C10022E7
:10324C007BFF7A0479391214827BFF7A0379F312AB
:10325C0014827520FF804F124B39EF24D0B4080034
:10326C00505090327C75F003A4C58325F0C5837350
:10327C0002329402329802329C0232A00232A40230
:10328C0032A80232AC0232B0B200801AB2018016FF
:10329C00B2028012B203800EB204800AB20580061C
:1032AC00B2068002B207E520FD7C00E4FF1247C3A2
:0232BC0080A5EB
:0132BE0022ED
:102C5F007BFF7A04797B1214827BFF7A0479B61298
:102C6F0014827555071249FA124214E4FB7901E4F4
:102C7F00FAE4FF74082FF8A6010FBF08F6124214EA
:102C8F007FF47E0112435AE925E0F90ABA08E20BF4
:102C9F00BB03DA1249FA1242147FF47E0112435A2F
:102CAF00E4FBE4FF124ADF8F087F01124ADF8F092E
:102CBF007F02124ADF8F0A7F03124ADF8F0B7F04D6
:102CCF00124ADF8F0C7F05124ADF8F0D7F06124AE3
:102CDF00DF8F0E7F07124ADF8F0F1242141249F354
:102CEF001242147FF47E0112435A0BBB03B4D290ED
:042CFF00D291D29408
:012D030022AD
:1028F6007BFF7A0479C01214827BFF7A0479B612C0
:1029060014821249FA75560F75680712462F123E41
:10291600CCE4F9752901E4F528E4FF74082FF8A63C
:10292600290FBF08F6123ECC7FF47E0112435AE50A
:102936002925E0F5290528E528D3940740DB09B9C0
:1029460003D11249FA123ECC7FF47E0112435AE4B7
:10295600F9E4FF124B918F087F01124B918F097F8B
:1029660002124B918F0A7F03124B918F0B7F041239
:102976004B918F0C7F05124B918F0D7F06124B9159
:102986008F0E7F07124B918F0F123ECC1249F31216
:102996003ECC7FF47E0112435A09B903B4D290D2D9
:0329A60091D29437
:0129A900220B
:103CC5007BFF7A0479FD1214827BFF7A0079461214
:103CD50014821249FA7F40124ACC20982F123927B4
:103CE5008F28E528F460F3E528124AD98F08E528DE
:103CF500540FFF124ADF8F0985080A85080C8508CD
:0F3D05000E85090B85090D85090F80CE024B39FC
:1046F2007BFF7A05792E1214827BFF7A05795B1291
:104702001482124B39AB07EB64036007AF03123A12
:034712008680EFAF
:014715002281
:103BD4007BFF7A057971121482124843123B2E122C
:103BE4003628920A300A08122831123628920A30EE
:103BF4000A097BFF7A02795E021482E4F52874785C
:103C04002528F582E43400F583E0FF60147BFF7A15
:103C14000579A78F351214820528E528D394274007
:013C2400DDC2
:013C2500227C
:1039DA007BFF7A0579AA1214827BFF7A0079461254
:1039EA00148220983F1248B7122E218F2B8E2A8DCF
:1039FA00298C28121F1F8F2F8E2E8D2D8C2C7BFF2A
:103A0A007A0579E2852B38852A378529368528353E
:103A1A008F3C8E3B8D3A8C391214827FE87E0312DA
:073A2A00435A80BE024B3934
:102BB5007BFF7A0579F3121482124A26AB07BB31E3
:102BC5000575281F800375287F7529F87BFF7A0610
:102BD50079101214827BFF7A0179C31214827BFF6C
:102BE5007A0179EE121482124B39AB07EB6453600C
:102BF50003BB7323751C28751D02751E04751B0107
:102C0500751A23751959751855AF29AE281234F15F
:102C15007FC87E0012435A7BFF7A007946121482E0
:102C25007BFF2098327F647E0012435AAF29AE287D
:102C3500123982E5186B60EA7BFF7A027911851AF1
:102C450035851936851837851C38851D39851E3A11
:0A2C5500121482AB1880CB024B3939
:103F9700BF3A0FE4F55DD21A7E29786AE4F608DEA7
:103FA700FC22301A2AEF640D6003BFFF0C746A25E8
:103FB7005DF8A607C21AD21722EFC394204010E576
:0F3FC7005DC394285009746A255DF8A607055D4F
:013FD60022C8
:0300230002465939
:0D465900C0E0C0D075D000C000C006C00792
:10466600309906C299D2188007AF99C298123F971F
:0B467600D007D006D000D0D0D0E0323A
:104862003019093018FDC2188F998012BF0A08301A
:0F48720099FDC29975990D3099FDC2998F9922C0
:094B4C007BFF7A06793E02148217
:094B55007BFF7A027966021482EA
:094B5E007BFF7A06794202148201
:094B67007BFF7A067946021482F4
:1049BC007BFF300A067A0179A880047A0179A61265
:0349CC0014822230
:0B4AF2007BFF7A0679498F35021482A1
:10188F00786BE6F52908E6F52AE529640D6042E54F
:10189F002AB40D02803BAF2A12475EAE07AF291262
:1018AF004952EF4EF529786DE6F52AB40D04C209B9
:1018BF008022786EE6640D60028016D209E52AB4A4
:1018CF003005E4F52A800DE52AB43105752A01802B
:1018DF0003024B5EE5291213CD194C00195D011956
:1018EF006E02197F0319900419A10519B20619C3C5
:1018FF000719D41019E51119F6121A07131A18142B
:10190F001A29151A3A161A4B171A5C201A6D211A32
:10191F007E221A8F231AA0241AB1251AC2261AD38F
:10192F00271AE2301AF1311B00321B0F331B1E3402
:10193F001B2D351B3C361B4B3700001B6230090932
:10194F00E52A24FF9280021B54A280021B5B300900
:10195F0009E52A24FF9281021B54A281021B5B30EE
:10196F000909E52A24FF9282021B54A282021B5B03
:10197F00300909E52A24FF9283021B54A283021B1C
:10198F005B300909E52A24FF9284021B54A28402CA
:10199F001B5B300909E52A24FF9285021B54A2859F
:1019AF00021B5B300909E52A24FF9286021B54A211
:1019BF0086021B5B300909E52A24FF9287021B541C
:1019CF00A287021B5B300909E52A24FF9290021BB4
:1019DF0054A290021B5B300909E52A24FF92910261
:1019EF001B54A291021B5B300909E52A24FF929236
:1019FF00021B54A292021B5B300909E52A24FF92B5
:101A0F0093021B54A293021B5B300909E52A24FFA2
:101A1F009294021B54A294021B5B300909E52A24FD
:101A2F00FF9295021B54A295021B5B300909E52A10
:101A3F0024FF9296021B54A296021B5B300909E504
:101A4F002A24FF9297021B54A297021B5B300909AD
:101A5F00E52A24FF92A0021B54A2A0021B5B3009AF
:101A6F0009E52A24FF92A1021B54A2A1021B5B309D
:101A7F000909E52A24FF92A2021B54A2A2021B5BB2
:101A8F00300909E52A24FF92A3021B54A2A3021BCB
:101A9F005B300909E52A24FF92A4021B54A2A40279
:101AAF001B5B300909E52A24FF92A5021B54A2A54E
:101ABF00021B5B300909E52A24FF92A6021B54A2E0
:101ACF00A6021B5B300908E52A24FF92A78076A2A5
:101ADF00A78079300908E52A24FF92B08067A2B069
:101AEF00806A300908E52A24FF92B18058A2B1809C
:101AFF005B300908E52A24FF92B28049A2B2804CDC
:101B0F00300908E52A24FF92B3803AA2B3803D3012
:101B1F000908E52A24FF92B4802BA2B4802E300945
:101B2F0008E52A24FF92B5801CA2B5801F30090852
:101B3F00E52A24FF92B6800DA2B6801030090BE57E
:101B4F002A24FF92B7124B55800CA2B7920A124962
:0F1B5F00BC8003124B677BFF7A06794F1214820A
:011B6E002254
:102F3C00786BE6F52B08E6F52908E6F52AE529B4C1
:102F4C000D04C2098023E52AB40D028007786EE6D1
:102F5C00640D6003024B5ED209AF2A12475EAE07C6
:102F6C00AF29124952EF4EF529E52B24CF601614E8
:102F7C00601F146028240370363009058529808071
:102F8C0022AF8080253009058529908016AF90806E
:102F9C00193009058529A0800AAFA0800D300908D9
:102FAC008529B0124B55800AAFB0124AF280031239
:0B2FBC004B677BFF7A06794F121482EE
:012FC70022E7
:1029AA00786BE6F52B08E6F52CE52B640D6068E5F7
:1029BA002CB40D028061AF2C12475EEFFD7C00AF94
:1029CA002B124952E4F529EF4DF52A786DE6F52BDD
:1029DA0008E6F52CE52B640D6005E52CB40D0280A4
:1029EA0036AF2B124952EFFDE52AFCAF2C12475E97
:1029FA00ECF529ED4FF52A786FE6F52B08E6F52C6C
:102A0A00E52BB40D04C2098023E52CB40D0280071E
:102A1A007871E6640D6003024B5ED209AF2C12474F
:102A2A005EAE07AF2B124952EF4EF52B30090E85D9
:102A3A002A82852983E52BF0124B55800B852A8241
:102A4A00852983E0FF124AF27BFF7A06794F121436
:012A5A0082F9
:012A5B002258
:1036ED00786CE6B40D028045786CE6FF12475E8F6C
:1036FD0059E55914601814601A14601C14602114D3
:10370D00602324057027756402755A08802275643C
:10371D000180087564028003756404755A10801069
:10372D007564028003756404755A148003024B5E40
:10373D00124A4812495EE4F563F567C215124B4C07
:01374D002259
:10348400786CE6640D605F08E6640D605908E664D4
:103494000D605308E6B40D02804C786CE6F55E08C6
:1034A400E6F55FE4F560FB7A00795E122A5C8F63CF
:1034B400E563D394134002802D786EE6FF12475ED5
:1034C4008F67E567D394034002801B786FE6FEB4F0
:1034D4003009C2157F0C124ABF800EEEB43107D2F8
:0D34E40015122EAF8003024B5E124B4C22DE
:103F54007F02AE070F746A2EF8E6FE640D6028E552
:103F640063C3955A50EC75F014E567A42563F58294
:103F7400E435F0F583E5822400F582E5833400F529
:103F840083EEF0056380CB1222EE301503122EAFC0
:033F9400024B4C91
:10471600786CE6FFB4300990D002E04410F08010C7
:10472600EFB4310990D002E054EFF08003024B5E03
:04473600124B4C22B4
:10473A00786BE6FF124A37EF24BE601424F2600A4F
:10474A0024FC600904700C0236ED023484023F54E2
:04475A0012471622CA
:0232BF00AC075A
:1032C1001249FA7B03E4FEAF030B746A2FF8E6FDA3
:1032D100640D603BBD2D0874082EF87640802DBD2D
:1032E100200874082EF8E4F68022BD2E11EED39446
:1032F1000040011E74082EF8E64480F6800EAF05EA
:1033010012475E124ADF74082EF8A6070E80B8BC79
:10331100300A123927AD07BFFF0780F6123927ADF2
:1033210007BDFF027D637BFF7A0679518D3502145B
:013331008219
:02374E00AE07C4
:103750001249FA7D03E4F9AF050D746A2FF8E6FC0F
:10376000AF050D746A2FF8E6FBEC640D601FEB6487
:103770000D601AAF0312475EAA07AF04124952EF59
:103780004AFFAA010974082AF8A60780CABE300AAF
:10379000123927AC07BFFF0780F6123927AC07BCE8
:0F37A000FF027C637BFF7A0679518C350214821D
:1042E000786BE6FF124A378F29E52964306005E5CF
:1042F00029B4311A786CE6FF124A37EF24B8600906
:1043000024FA700DAF290232BFAF2902374E124B8B
:014310005E4E
:014311002289
:103C2600786BE6F55E08E6F55FE4F560FB7A007909
:103C36005E122A5CEF25E0F529786DE6F55E08E66A
:103C4600F55F7B007A00795E122A5C7C017D2C127E
:103C560013878E2A8F2BE5296006E52B452A7003EC
:0F3C6600024B5EAD2BAC2AAF29124171124B4CB1
:013C7500222C
:1041A90090D001E054F0F529E4F52AE5297BFF20B8
:1041B900E4067A0179A880047A0179A6121482E5C5
:1041C90029C313F529052AE52AD3940340DD7BFF8A
:0741D9007A06794F021482FF
:10401500786BE6B40D151242AE7BFF7A06795885AA
:104025001A35851936851837021482124946EF4E1E
:10403500F51A786E124948EF4EF51978701249480D
:0B404500EF4EF518120003124B4C2246
:103FD700786BE6B40D151242AE7BFF7A06795885E9
:103FE7001C35851D36851E37021482124946EF4E51
:103FF700F51C786E124948EF4EF51D787012494846
:0E400700EF4EF51E124B11120006124B4C220A
:1030D900786BE6F52908E6F52AE529640D6036E5F9
:1030E9002AB40D02802FAF2A12475EAE07AF29120C
:1030F9004952EF4EF52B786DE6F52908E6F52AE5F4
:1031090029640D6005E52AB40D04C209801C786F95
:10311900E6640D6003024B5ED209AF2A12475EAE28
:1031290007AF29124952EF4EF52930090DE529FD5E
:103139007C00AF2B124824024B4CAF2B1243D38F88
:0D314900297BFF7A067969852935121482E9
:013156002256
:094B70007BFF7A067970021482C1
:1047E400AE07786DE6FF12475E8F5608E6FF124764
:1047F4005E8F68BE3305124605800312462F024BB6
:014804004C67
:02386D00AE07A4
:10386F001249FA7D03E4FCAF050D746A2FF8E6FFE9
:10387F00640D6039BF2D0874082CF87601802BBFBA
:10388F00200874082CF8E4F68020BF2E11ECD39496
:10389F000040011C74082CF8E64480F6800C124797
:1038AF005E124B9174082CF8A6070C80BABE330534
:0B38BF00123E878003123ECC024B4CEF
:023D1400AE07F8
:103D16001249FA7D03E4F9AF050D746A2FF8E6FC43
:103D2600AF050D746A2FF8E6FBEC640D601FEB64BB
:103D36000D601AAF0312475EAA07AF04124952EF8D
:103D46004AFFAA010974082AF8A60780CABE3305E5
:0B3D5600123E878003123ECC024B4C53
:10405000786BE6FF124A378F29E52964316005E560
:1040600029B43323786CE6FF124A37EF24B8601284
:1040700024FA600924FB7012AF290247E4AF290239
:0A408000386DAF29023D14124B5EAB
:01408A002213
:10492F00786DE6BF3308FF12475E8F5C8006FF127B
:07493F00475E8F55024B4C4F
:0238CA00AE0747
:1038CC001249FA7D03E4FCAF050D746A2FF8E6FF8C
:1038DC00640D6039BF2D0874082CF87640802BBF1E
:1038EC00200874082CF8E4F68020BF2E11ECD39439
:1038FC000040011C74082CF8E64480F6800C12473A
:10390C005E124ADF74082CF8A6070C80BABE330589
:0B391C001241E08003124214024B4CE9
:023D6100AE07AB
:103D63001249FA7D03E4F9AF050D746A2FF8E6FCF6
:103D7300AF050D746A2FF8E6FBEC640D601FEB646E
:103D83000D601AAF0312475EAA07AF04124952EF40
:103D93004AFFAA010974082AF8A60780CABE330598
:0B3DA3001241E08003124214024B4C5E
:10408B00786BE6FF124A378F29E52964316005E525
:10409B0029B43323786CE6FF124A37EF24B8601249
:1040AB0024FA600924FB7012AF2902492FAF2902B1
:0A40BB0038CAAF29023D61124B5EC6
:0140C50022D8
:10368B00124843786BE6FF124A37BF3305123ADB19
:10369B00800ABF3105123B2E80028013123628920E
:1036AB000930090812283112362892093009030211
:1036BB004B5EE4F52974782529F582E43400F58313
:1036CB00E0FF60147BFF7A0579A78F351214820512
:1036DB0029E529D3942740DD7BFF7A06794F121415
:0136EB00825C
:0136EC0022BB
:1035C200786BE6FF124A378F31E531B43313124874
:1035D2009D122D938F2C8E2B8D2A8C29121D6F807C
:1035E20016E531B4311B1248B7122E218F2C8E2BC7
:1035F2008D2A8C29121F1F8F308E2F8D2E8C2D809D
:1036020003024B5E7BFF7A06797E852C38852B3749
:10361200852A3685293585303C852F3B852E3A858E
:053622002D3912148295
:013627002280
:102B0A00786BE6F52D64316008E52D643360028048
:102B1A0046786CE6F52B08E6F52CE52B640D600586
:102B2A00E52CB40D028030AF2C12475EAE07AF2BF6
:102B3A00124952EF4EF529786EE6F52B08E6F52C88
:102B4A00E52BB40D04C2098023E52CB40D028007DD
:102B5A007870E6640D6003024B5ED209AF2C12470F
:102B6A005EAE07AF2B124952EF4EF52A300920E527
:102B7A002DB4310CE52AFD7C00AF291247C3800A27
:102B8A00E52AFD7C00AF291247A2124B558012E5B7
:102B9A002DAF29B4310512490180031248EA124ABD
:0A2BAA00F27BFF7A06794F121482C5
:012BB40022FE
:1037AF00786BE6FF124A378F29E529643370237F40
:1037BF003A123A31752A02746A252AF8E6F52BB4C3
:1037CF000D077F0D123A318027AF2B123A31052AA0
:1037DF0080E5E529643170247F3A123A86752A0212
:1037EF00746A252AF8E6F52BB40D087F0D123A8678
:0F37FF00024B4CAF2B123A86052A80E4124B5E28
:01380E002297
:10276B0090D0037482F090D002E04450F0D219D292
:10277B00ACD2AFE4F55DD21A7F29786AE4F608DFB4
:10278B00FC7F293017FDC217124AFD786AE6FF124B
:10279B004A37EF1213CD280A30280F31281432286C
:1027AB001933281E3428233528283627F1422800D0
:1027BB004428054527E74C27D85027DD5227EC53F3
:1027CB0027FB5427F65727E2580000282B12188FA7
:1027DB00804E122F3C80491229AA804412473A801E
:1027EB003F1242E0803A123C2680351241A98030DC
:1027FB00124015802B123FD780261230D980211220
:10280B004B70801C124050801712408B8012123676
:10281B008B800D1235C28008122B0A80031237AF42
:06282B00124B8902278E0A
:1033A300D299C2B41220CF123F11BF3A0312276B36
:1033B30090D0037482F090D002E04450F0C219120E
:1033C3004AFD1240C68E278F287526017BFF7A0699
:1033D300798F1214820526E526D3941640EE7BFFDF
:1033E3007A0679911214827BFF7A0679B78527359D
:1033F3008528368557378558381214827BFF7A061D
:1034030079CF1214827BFF7A0679EB121482024B76
:01341300397F
:1023E700E4F526D2093009637BFF7A0279A7121434
:1023F700827BFF7A0679FE1214827BFF7A077922A5
:102407001214827BFF7A0779481214827BFF7A07BE
:10241700796D1214827BFF7A0779951214827BFFFC
:102427007A0779B41214827BFF7A0779D51214825E
:102437007BFF7A0779FD1214827BFF7A08792112D4
:1024470014827BFF7A08792B121482C209E5266071
:1024570007F527E4F5268008124B39124A378F27EC
:10246700E52724AF606E2420B40700505B902482D8
:1024770075F003A4C58325F0C5837302249702244E
:102487009F0224A70224AF0224B70224BF0224C755
:10249700D2091225CF0223ECD20912355B0223ECB5
:1024A700D20912324C0223ECD209122C5F0223EC20
:1024B700D2091228F60223ECD209123CC50223ECFA
:1024C700D2091246F20223EC7BFF7A0879371214FD
:0424D700820223EC6E
:0124DB0022DE
:1024DC00E4F526D2093009637BFF7A0279A712143E
:1024EC00827BFF7A0879391214827BFF7A0879583B
:1024FC001214827BFF7A0879641214827BFF7A08AB
:10250C0079701214827BFF7A08797C1214827BFF1B
:10251C007A0879881214827BFF7A087994121482D3
:10252C007BFF7A0879A01214827BFF7A087921123A
:10253C0014827BFF7A08792B121482C209E526607B
:10254C0007F527E4F5268008124B39124A378F27F6
:10255C00E52724AF606C2420B407005059902577F0
:10256C0075F003A4C58325F0C5837302258C022561
:10257C009302259A0225A10225A80225AF0225BAAD
:10258C00D209E4F5598021D209755901801AD20972
:10259C007559028013D209755903800CD2097559EB
:1025AC00048005D2097559051221ED0224E1D209E6
:1025BC001246CD0224E17BFF7A087937121482028D
:0225CC0024E108
:0125CE0022EA
:102D0400E4F526D20930093F7BFF7A0279A7121431
:102D1400827BFF7A0879B61214827BFF7A0879E005
:102D24001214827BFF7A0879F81214827BFF7A09E5
:102D340079131214827BFF7A0879211214827BFFA3
:102D44007A08792B121482C209E5266007F527E474
:102D5400F5268008124B39124A378F27E52724CEEF
:102D6400601214601624E2602524207015D2091222
:102D74003BD48091D2091239DA808AD209122BB558
:0E2D840080837BFF7A087937121482022D09B2
:012D9200221E
:101B6F00E4F5241233A3D208200803021C5E7BFF86
:101B7F007A0279A71214827BFF7A09792A121482CA
:101B8F007BFF7A0979671214827BFF7A0979A41295
:101B9F0014827BFF7A0979D01214827BFF7A0A793B
:101BAF000B1214827BFF7A0A79461214827BFF7A1A
:101BBF000A79811214827BFF7A0A79B51214827B1B
:101BCF00FF7A0A79E11214827BFF7A0B790D1214D6
:101BDF00827BFF7A0B79391214827BFF7A0B79742F
:101BEF001214827BFF7A0B79AF1214827BFF7A0B70
:101BFF0079E31214827BFF7A0C79171214827BFF20
:101C0F007A0C794B1214827BFF7A0C797F12148233
:101C1F007BFF7A0C79BA1214827BFF7A0C79F5125A
:101C2F0014827BFF7A0D79301214827BFF7A0D7943
:101C3F006B1214827BFF7A0D79851214827BFF7AE7
:101C4F000D799A1214827BFF7A08792B121482C2B3
:101C5F0008E5246007F525E4F5248008124B3912B6
:101C6F004A378F25E5251213CD1CBB311CC3321CFF
:101C7F00CB331CD3341CDB351CE3361CEB371CF386
:101C8F00381CFB391D03411D0B421D13431D1B4403
:101C9F001D23451D2B461D33471D3B481D43491D25
:101CAF004B581D53591D5B5A00001D63D208124239
:101CBF007B021B77D208123DAE021B77D20812416E
:101CCF0038021B77D208123157021B77D208124AFB
:101CDF0068021B77D208122FC8021B77D208123C5A
:101CEF0076021B77D208123332021B77D2081230DA
:101CFF0053021B77D208123B81021B77D20812497D
:101D0F0096021B77D2081249A9021B77D208123DFF
:101D1F00F9021B77D20812496F021B77D208124AB9
:101D2F0004021B77D208124A15021B77D208123110
:101D3F00D3021B77D208123414021B77D208122356
:101D4F00E7021B77D2081224DC021B77D208122D70
:101D5F0004021B777BFF7A087937121482021B77F4
:100DFA000210D8E86480F8E933E83360110460F03F
:100E0A00ED33EC337009E8FCE9FDEAFEEBFF22045E
:100E1A0060DED3EB9FEA9EE99DE8C2E78CF0C2F759
:100E2A0095F0400CE8CCF8E9CDF9EACEFAEBCFFB25
:100E3A001210A385D0F05804700320D5B3E80470CB
:100E4A00075002B2D50210E292D5EC0460F7E4CC66
:100E5A00C0E0C398F8603B94186008400DD0E0FBEE
:100E6A000210BAE4FBFAC9FC8028E830E406E4C9B7
:100E7A00FBE4CAFCE830E305E4C9CACBFCE8540742
:100E8A006010F8C3E913F9EA13FAEB13FBEC13FC4D
:100E9A00D8F130F52FC3E49CFCEF9BFFEE9AFEEDF0
:100EAA0099FDD0E0FBEF4E4D4C701222DB0302108D
:100EBA00DFEC2CFCEF33FFEE33FEED33FDED30E7D4
:100ECA00EB0210BAEF2BFFEE3AFEED39FDD0E0FB54
:100EDA0050130BBB00030210E2ED13FDEE13FEEFFD
:080EEA0013FFEC13FC0210BA27
:100EF200EC4D6011E8497017ED33EC3304600DE4FA
:100F0200FCFFFEFD22E933E8330470F80210D81228
:100F120010A358046009E4CC248150062850090229
:100F220010E22840030210DFC0E0EB4A7044B980AF
:100F320006D0E0FB0210CEEF4E701CBD8008EBFF26
:100F4200EAFEE9FD80EBE98DF0A4FEE5F0020FDB9D
:100F5200E9CDF9EAFEEBFFEF89F0A4FCE5F0CE89DA
:100F6200F0A42EFFE435F0CD89F0A42DFEE435F097
:100F72008067EF4E7005BD80D780C3EF8BF0A4ACC5
:100F8200F0EE8BF0A42CFCE435F0F8EF8AF0A42C00
:100F9200E5F038FCE433CB8DF0A42CFCE5F03BF813
:100FA200EE8AF0A42CFCE5F038F8E433CF89F0A403
:100FB2002CFCE5F038CF3400CE89F0A42FFFE5F009
:100FC2003EFEE433C98DF0A42EFEE5F039CD8AF061
:100FD200A42FFFE5F03EFEE43DFD33D0E0FB5007D9
:100FE2000BBB000F0210E2EC2CFCEF33FFEE33FEE2
:060FF200ED33FD0210BA10
:100FF80074F8CC6480CCC86480C8F582046043C3AC
:10100800EB9FF5F0EA9E42F0E99D42F0E89C45F03E
:1010180060305018E5825FFFE582F42B5582FB5063
:10102800210ABA001D09B90019088016E5825BFB80
:10103800E582F42F5582FF50090EBE00050DBD0054
:10104800010CC3EB9FF5F0EA9E42F0E99D42F0E8FF
:0D1058009C45F06007CC4820E701B3EC2276
:1010650075F020800E75F010800575F0087D007E06
:10107500007F003392D530D503121399EC3340101D
:10108500EF33FFEE33FEED33FDEC33FCD5F0ED220F
:0E109500E5F0247EA2D513CC92E7CDCEFF224B
:10142000E5492435F8E6054922783230120278354C
:10143000E475F0011213BD02132F200BEB7F2ED2A7
:101440000B8018EF540F2490D43440D4FF300F0B8E
:10145000EF24BFB41A0050032461FFE54A6002156F
:101460004A054DE54D7002054C30120D7832E47599
:10147000F0011213BDEF0213750248627403D21219
:101480008003E4C212F5498B328A338934E4F54A89
:10149000F54CF54DE54A60077F2012145B80F57529
:1014A0004BFFC20CC20BC20DC20EC210C211C2133E
:1014B000121429FF700D3012057F0012146CAF4D0D
:1014C000AE4C22B4255FC2D5C20F121429FF24D01E
:1014D000B40A00501A75F00A784A30D50508B6FFEC
:1014E0000106C6A426F620D5047002D20E80D924A7
:1014F000CFB41A00EF5004C2E5D20F021759D20C34
:1015000080C6D20B80C0D20D80BCD2D580BAD2109A
:1015100080B47F2012145B200D077401B54A00408F
:10152000F1121420FF12145B021494D213D2118012
:1015300095121420FB121420FA121420F94A4B7051
:101540000679507A187BFF200D2EE54A602A7E002E
:101550008E8275830012134860060EEE654B70F0A4
:10156000C2D5EBC0E0EAC0E0E9C0E0EE1217B9D0A6
:10157000E0F9D0E0FAD0E0FB12132FFF60AAEBC035
:10158000E0EAC0E0E9C0E012145BD0E02401F9D049
:10159000E03400FAD0E0FBE54B0460DCD54BD980A9
:1015A00087D20D80A212179C60F7E54B70010412E0
:1015B00010EDA94B600DE54B600914F54B12184373
:1015C000EF60F3EA30E702F404C3995077EAF425B8
:1015D0004B0430E701E404F54B800D12179C60C109
:1015E000EA054B254B1210EDEA7848F630E701E4A6
:1015F000254B04D54B04201001141217B9E4C0E0A8
:101600001218437848E6601320E70714F6121443D3
:10161000802204F6D0E014C0E07F00121443E54BB2
:10162000600712143A154B800B30100312143AD095
:10163000E0021494D0E00480C512179C60A0E54B32
:10164000041210ED7848EAF6E54B20100260010420
:0516500024041217B98B
:1016550074FF04C0E0121843121443E54B20100236
:10166500600312143AD0E0B54BE87F4512144D786B
:1016750048E67F2B30E7047F2DF404C0E012145BAD
:10168500D0E075F00A84C0F0121444D0E01214447E
:10169500021494791080027908C211C2138008D20D
:1016A500D5790A8004790AC2D5E54B047002F54B59
:1016B500E4FAFDFEFF121420FC7B08200C13121423
:1016C50020FD7B10300B0A121420FE121420FF7B24
:1016D50020EC3382D592D55013C3E4300B069FFF1F
:1016E500E49EFEE4200C039DFDE49CFCE4CBF8C2E3
:1016F5000CEC700CCFCECDCCE824F8F870F3801745
:10170500C3EF33FFEE33FEED33FDEC33FCEB33FB80
:10171500994002FB0FD8E9EB300C05F8D0E0C4483E
:10172500B20CC0E00AEC4D4E4F78207B0070C2EA47
:10173500B54B0040BCC0E01217BBD0F0D0E0200C88
:1017450004C4C0E0C4B20CC0F0121444D0F0D5F00B
:10175500EB0214941213CD15315316985815024CFB
:1017650014FE42169C4F16A44416A4491517431699
:10177500AA5515DB4616394515A5471870501506A7
:101785002D150A2E152D2B150E23152B2018592A2C
:1017950014C64800001525E54BB4FF03754B06122A
:1017A5001420FC121420FD121420FE121420FF78C0
:1017B5004102111C790AA2D5200E14301009B91066
:1017C500020404B9080104A2D52011025001042025
:1017D5000D68920DB54A005034C0E07F20300E19D7
:1017E5007F30A20D72117210500F121812C20DC265
:1017F50011C210C2137F30800F301003E9C0E01210
:10180500145B301003D0E0F9D0E0B54ACC301017A6
:101815007F30B9100C12145B7F58300F077F78802A
:1018250003B9080312145B300D057F2D02145B7F8D
:10183500202013F87F2B2011F322920D80CF7F00FB
:10184500B4070050052441F8E6FF22286E756C6C3C
:101855002900D20C121420300CF8C20C784A30D56D
:101865000108F60214C62D504349581214202403CA
:10187500B405004001E490186B9312144C743A12AD
:0A188500144CD20E754A04021698A6
:1010A300E9D2E7C933E833F892D5EDD2E7CD33EC93
:0710B30033FC5002B2D5220C
:1010BA00EC30E7100FBF000C0EBE00080DBD000497
:1010CA000BEB6014A2D5EB13FCED92E7FD2274FF43
:1010DA00FCFDFEFF22E480F8A2D574FF13FC7D809C
:0310EA00E480EFB0
:1010ED00F920E72824F950037907E4F42402FB18CA
:1010FD00DBFDE624FB5014E9600DE4F618E604F67A
:0F110D00B40A08E4F6D9F57401F60A22C2D52215
:10111C00ED33EC3392D5FA602AB4FF33EDC2E77BA2
:10112C00FF60067A117941E4227A11794A20D504BC
:10113C007A117945224E614E002B494E46002D49BD
:10114C004E4600E47A08F608DAFC7B00740722E8C5
:10115C00C0E0ECC0E0EDC0E0EEC0E0EFC0E0EA754E
:10116C00F010A4CAABF075F04DA42BFBE435F0FCE9
:10117C00EA2410FAEB34C5FBEC34D9FCEDC2E7FFE2
:10118C0075F056A4F42411C5F0F434C58FF0A42ADC
:10119C00E5F03BE43CF620E7141212EFD0E0FFD070
:1011AC00E0FED0E0FDD0E0FC1212228014F4041218
:1011BC0012EFD0E0FFD0E0FED0E0FDD0E0FC120E4C
:1011CC00F2D0E0F8E6FAEDD2E7CD33EC332482FB33
:1011DC00E4C3CF33CFCE33CECD33CD33DBF37B076C
:1011EC0075F00A846004F6081B0AE5F0F6088FF027
:1011FC00740AA4FFACF08EF0740AA42CFEACF05070
:10120C00010C8DF0740AA42CFDE435F0F608DBDE3D
:03121C0074072232
:10121F000210E2EC5D046005E8590470030210D877
:10122F001210A3580460F6EC4860F2EC7004FDFE57
:10123F00FF22C860DB2481C85009C39860025006A2
:10124F000210DF9850CAF582E9294B4A7005AB822C
:10125F000210CE75F0007C1A7880C3EF9BEE9AEDEA
:10126F0099400DC3EF9BFFEE9AFEED99FDE842F01A
:10127F00DC23ACF0D0E0FFD0E0FED0E0FDAB82206D
:10128F00E7101BEB60BAEC2CFCEF33FFEE33FEEDF7
:10129F0033FD0210BAE803F830E705C0F075F0002F
:1012AF00EF2FFFEE33FEED33FD40B830E7C280AADB
:1012BF003F8000004120000042C80000447A000037
:1012CF00461C400047C35000497424004B189680B9
:1012DF004CBEBC205A0E1BCA6753C21C749DC5AEB0
:1012EF00FB60065407601C232312131DEB54386058
:1012FF0009121309121318120EF2ECF8EDF9EEFAA7
:10130F00EFCB22EB12131880F1543803241C9012E8
:10131F00BFFE93FC0EEE93FD0EEE930ECE93FF22C7
:03000000024AE6CB
:0C4AE600787FE4F6D8FD758192021B6F0A
:10132F00BB010689828A83E0225002E722BBFE02BC
:09133F00E32289828A83E49322EF
:10134800BB010CE58229F582E5833AF583E022505A
:1013580006E92582F8E622BBFE06E92582F8E222A4
:0D136800E58229F582E5833AF583E49322BE
:10137500BB010689828A83F0225002F722BBFE0157
:02138500F32251
:10138700EF8DF0A4A8F0CF8CF0A428CE8DF0A42E7A
:02139700FE2234
:0E139900C3E49FFFE49EFEE49DFDE49CFC2265
:1013A700EB9FF5F0EA9E42F0E99D42F0EC6480C8BD
:0613B70064809845F0225D
:1013BD00FAE6FB0808E6F925F0F618E6CA3AF62231
:1013CD00D083D082F8E4937012740193700DA3A3AF
:1013DD0093F8740193F5828883E4737402936860C3
:0613ED00EFA3A3A380DFC3
:1013F300D083D082F8E4937012740193700DA3A389
:1014030093F8740193F5828883E473740293B5F0BF
:0D141300067403936860E9A3A3A3A380D827
:0A4B39003098FDAF99C2987E00226B
:104A2600101B0B124B39BF0D027F0A024862AF6999
:014A3600225D
:104A3700EFC39461400AEF947B5005EF24E0FF2217
:014A4700224C
:102A5C008B2C8A2D892EAB2CAA2DA92E12132FFF6D
:102A6C001249CF500D7401252EF52EE4352DF52D80
:102A7C0080E4D209AB2CAA2DA92E12132FFF642BA4
:102A8C006004EFB42D1BAB2C052EE52EAA2D700285
:102A9C00052D14F912132F642D6003D38001C392FA
:102AAC0009E4F52FF530AB2CAA2DA92E12132FFF0C
:102ABC00124A785036AB2CAA2DA92E12132FFF33A5
:102ACC0095E0FEEF24D0FBEE34FFFAAE2FAF307C56
:102ADC00007D0A121387EF2BF530EE3AF52F7401B7
:102AEC00252EF52EE4352DF52D80BB300906AE2FA5
:0E2AFC00AF308009C3E49530FFE4952FFE2231
:0F4A7800EFC394304007EF943A50028001C322FD
:1049CF00EFC394094005EF940E4003BF2003D3803B
:0349DF0001C322EF
:00000001FF
